:1000000012C01895189518951895189518953DC310
:100010001895189518951895189518951895189578
:100020001895189518958FED8DBFC0ECE6EA4E2E09
:10003000DD275D2EEEE7F0E0A0E6B0E0A89584B7FE
:10004000082E877F84BF88E1992781BD91BD8827CD
:100050008D933197E9F78FE889B980E082B988E11B
:100060008AB966248EE083B97894579A8D9A8E9ACD
:1000700068D29698A8E6BA93AA9345D22296969A01
:10008000009168000A3009F006C081E8A2D25FD270
:1000900081E89FD235C2009168000F3081E009F0FD
:1000A00080E08F93009168000B3081E009F080E0E0
:1000B0009F91892B882309F45AC0A5E610D380E0CC
:1000C00088D288E586D280E084D280E082D28BEB31
:1000D00080D284E690E0B1D249D2ACE68C93009114
:1000E0006C00013009F003C047D2AFE68C9382E385
:1000F00090E0A3D23BD2ACE68C9300916C0001302F
:1001000009F034C039D2A0E78C93009168000B301D
:1001100009F01AC000916F0043E00423ABE60C9392
:10012000ABE68C918F5F8C93ABE68C9183708C9354
:10013000AFE68C918C7F8C9300916F0040916B00A7
:10014000040FAFE60C9306C0AFE68C918C9390E859
:1001500089278C9380E03DD288E53BD231E0AFE641
:1001600033D231E0A0E730D28CEB33D2C9C1009159
:1001700068000C3009F04EC0A5E6B1D280E029D26B
:1001800089E727D280E025D280E023D28BEB21D2F1
:1001900084E690E052D2EAD1A8E68C930091680000
:1001A000013009F003C0E8D1AFE68C9382E390E020
:1001B00044D2DCD1A8E68C9300916800013009F0AC
:1001C00028C0DAD1A0E78C9300916F0043E00423AC
:1001D000ABE60C93ABE68C918F5F8C93ABE68C9186
:1001E00083708C93AFE68C918C7F8C9300916F0021
:1001F00040916B00040FAFE60C9380E0EAD189E7F1
:10020000E8D131E0AFE6E0D131E0A0E7DDD18CEB21
:10021000E0D176C1009168000E3009F0C1C0A8E6B7
:10022000BA93AA9370D12296009168000D3009F01C
:1002300060C0A8E6BA93AA9366D12296A5E64FD2EB
:1002400080E0C7D184D183E0C4D184E690E0F5D1C9
:100250008DD1AFE68C9300916F00013009F048C05A
:100260008BD1AFE68C9388D1A0E78C9385D1A1E7A1
:100270008C9382D1A2E78C937FD1A3E78C930091DA
:10028000680045E055D2A4E74C93E4E7F0E0A19084
:10029000E0E0F0E0EA0DAFE67BE72FD2E4E7F0E044
:1002A000A190E1E0F0E0EA0DA0E77BE726D2E4E7E9
:1002B000F0E0A190E2E0F0E0EA0DA1E77BE71DD2DB
:1002C000E4E7F0E0A190E3E0F0E0EA0DA2E77BE7ED
:1002D00014D2A3E78C918F708C93E4E7F0E0A190A7
:1002E000E4E0F0E0EA0DA3E77BE707D22AD129D1C9
:1002F00056C00091680045E01BD2A4E74C93E4E7A8
:10030000F0E0A190E0E0F0E0EA0DAFE607D2E4E72C
:10031000F0E0A190E1E0F0E0EA0DA0E7FFD1E4E732
:10032000F0E0A190E2E0F0E0EA0DA1E7F7D1E4E728
:10033000F0E0A190E3E0F0E0EA0DA2E7EFD1E4E71E
:10034000F0E0A190E4E0F0E0EA0DA3E7E7D131E0CE
:10035000AFE63AD131E0A0E737D131E0A1E734D1BF
:1003600031E0A2E731D181E034D184E690E065D17B
:1003700031E0A3E729D1EBD087E02BD184E690E0F0
:100380005CD131E0AFE620D131E0A0E71DD131E012
:10039000A1E71AD131E0A2E717D181E01AD1B0C0AC
:1003A000009168000D3009F03CC0A8E6BA93AA930A
:1003B000AAD0229600916800073009F004C081E0BD
:1003C00080936F0027C000916800083009F004C0D6
:1003D00080E080936F001EC000916800043009F037
:1003E00004C084E080936F0015C000916800053060
:1003F00009F004C088E080936F000CC00091680091
:10040000063009F004C083E080936F0003C082E0EF
:1004100080936F0031E0AFE6D7D099D087E0D9D094
:100420006FC0809168008093690082E080936F00C4
:1004300000916F00063010F009F00CC080E0AFE6CC
:10044000AD90A8E6AA0D8C93AFE68C918F5F8C934C
:1004500008F4EECF82E080936F0000916F000630C9
:1004600010F009F019C0A8E6BA93AA934CD02296CE
:10047000009168000A3008F008C080916800AFE67B
:10048000AD90A8E6AA0D8C9301C006C0AFE68C9192
:100490008F5F8C9308F4E1CF0091690040E148D16F
:1004A000AFE64C9300916F0040916A00040FAFE6F5
:1004B0000C9331E0AFE688D000916B0040E138D179
:1004C000AFE64C9300916F0040916C00040FAFE6D3
:1004D0000C9331E0AFE678D000916D0040E128D177
:1004E000AFE64C9300916F0040916E00040FAFE6B1
:1004F0000C9331E0AFE668D080E06BD081E069D04A
:10050000B8CDF894FFCF81E0A7D070D0A881B98191
:100510000C93A881B9810C91003109F402C011D06B
:1005200001C0F3CFECE5F5E0A881B9818C91992762
:10053000AA81BB81A7D081E0481A8827580A229651
:100540000895959884E690E078D0959A089580E093
:1005500040D080E03ED080E03CD008950102030A04
:100560000405060B0708090C0D000E0F80916700AB
:10057000882309F081E0089580916700882309F4B9
:1005800008950F929F93AF93BF937F9380916700DD
:100590008823E1F3F894809167008A95809367003F
:1005A00090916500A0E6A90F0024B01D8C91939551
:1005B000953009F499279093650078947F91BF91C5
:1005C000AF919F910F9008958D9103D03A95E1F7E7
:1005D00008955D9BFECF8CB908953197F1F708958A
:1005E000689462F80895E89462F8089500E18FEF46
:1005F00088BB8FE087BB80EF88BB82E38A95F1F7E9
:10060000B49B00E0B59B04E0B69B08E0B79B0CE010
:1006100080EF87BB8FE088BB82E38A95F1F788275C
:10062000B09B80E0B19B81E0B29B82E0B39B83E012
:10063000080F88EC90E001D00895EF93FF93EE2728
:10064000E82BE92B31F0EDECFAE03197F1F7019767
:10065000D1F7FF91EF9108955A924A92480E882758
:10066000581E0895C89531960020089591E005C060
:1006700092E003C094E001C098E0F4DF0D929A95F7
:10068000E1F70895E80FF91FF1CF7F930F93AF9330
:10069000BF938F939F938FB78F938091670005E0EF
:1006A000081B19F49CB19CDF11C000916600A0E604
:1006B00077279CB1A00FB71F9C9383958093670009
:1006C0000395053009F40027009366008F918FBFD2
:1006D0009F918F91BF91AF910F917F9118956FB7B7
:1006E000F894882793E08D939A95E9F76FBF089562
:1006F000E199FECFEEBB3196089591E001C092E002
:100700007B3751F47FB7F894F3DF8D918DBBE29A7C
:10071000E19A9A95C9F77FBF7727089591E001C0C4
:1007200092E0E6DFE09A8DB38D939A95D1F7089524
:10073000FF935527F8E0469508F4500F57954795D5
:08074000FA95D1F7FF9108952D
:00000001FF
